:03800000028100FA
:06800B00438CDC05083285
:2081000075811B90F000E4F0438901D2AFD2A9D28C128117021954128290128132128547F3
:20812000F5131284361284E21284FC12834102811D2212855974D075F000C0E0C0F0128549
:208140006E15811581740775F000C0E0C0F012856E15811581749075F000C0E0C0F01285D4
:208160006E158115811285662212855974D075F000C0E0C0F012856E15811581740075F053
:2081800000C0E0C0F012856E1581158112856612855974D175F000C0E0C0F012856E1581DC
:2081A00015817400F51B7400F509E50975F0007B067C0012884045F070030281E28008E58F
:2081C0000904F5091480E3E509790B7A0075F000128796C001C002128598D007D000F6024C
:2081E00081BF7401F51BE509790B7A0075F000128796C001C002128598D007D000F6128554
:2082000066743275F089C0E0C0F0740475F000790B7A00128796E775F000C0E0C0F07405F5
:2082200075F000790B7A00128796E775F000C0E0C0F0740675F000790B7A00128796E775A8
:20824000F000C0E0C0F0740275F000790B7A00128796E775F000C0E0C0F0740175F00079E7
:208260000B7A00128796E775F000C0E0C0F0740075F000790B7A00128796E775F000C0E0BC
:20828000C0F0740775F0001285287FF21287802212855974D075F000C0E0C0F012856E15E0
:2082A000811581740075F000C0E0C0F012856E15811581740075F000C0E0C0F012856E150A
:2082C000811581743075F000C0E0C0F012856E15811581741275F000C0E0C0F012856E15A8
:2082E000811581740375F000C0E0C0F012856E15811581742575F000C0E0C0F012856E15A2
:20830000811581740775F000C0E0C0F012856E15811581740075F000C0E0C0F012856E15A2
:2083200081158112856622128169229088AAE0A3F5F0E0C5F0C0E0C0F01285CB158115814C
:2083400022E51375F0007B0D7C0012882D45F0700302836C9088A8E0A3F5F0E0C5F0C0E0DD
:20836000C0F01285CB1581158112832B2205810581058105810581740075F00078FD128758
:2083800074F608A6F078FD128774E60886F07B027C0012880D45F070030283DF801678FD38
:2083A000128774E60886F01287F318F608A6F01287FC80D178FD128774E60886F079FA12C3
:2083C0008779128796C001C0021285F6C0E0C0F01285DE15811581D007D000F602839E7835
:2083E000FD128774E60886F079FA1287791287967400F7740075F00079FA12877912879663
:20840000E7C394301287A67B0412879D1287E2C0E0C0F0740175F00079F8128779128796A3
:20842000E7C39430D004D0034BC5F04CC5F01287A67FFB02878FE51375F0007B747C00127B
:20844000882D45F070030284E1745275F089C0E0C0F01285CB1581158112836DF516743A0B
:2084600075F000C0E0C0F01285DE1581158112836DF515743A75F000C0E0C0F01285DE15AD
:2084800081158112836DF51412855974D075F000C0E0C0F012856E15811581740075F000C7
:2084A000C0E0C0F012856E15811581E51475F000C0E0C0F012856E15811581E51575F000FD
:2084C000C0E0C0F012856E15811581E51675F000C0E0C0F012856E158115811285661283A8
:2084E0002B22E51375F0007B2F7C0012882D45F070030284FB12832712832B22E51375F0C1
:20850000007B3F7C0012882D45F070030285279088ACE0A3F5F0E0C5F0C0E0C0F01285CB95
:208520001581158112832B2223F42581F812887E12860612887E0285D578FB128774E630B8
:2085400099FDC299F5992274FFF5F030980A3098FDC298E59975F00022D2B41285BEC2B4DB
:208560001285C4C29022C2B41285BED2B42278FB128774E67F0830E704D2B48002C2B41221
:2085800085BE23C290DFEFD2B41285BE30B4001285C4C2901285C4227F087400D2B4128554
:2085A000BEA2B433C290DFF6C0E0D2B4E51BB40002C2B41285BEC290D0E075F00022D290BB
:2085C0003090FD220022000000002278FB1287748682088683E0602D1285E4A380F778FB6A
:2085E000128774E63099FDC299F599B40A17740D80F2E430980C3098FDC298E599B40D02F9
:20860000740A75F0002212874D868208868308E4FEFFE0700612874DE4F022B42551A3E08E
:20862000B42D05430780A3E0B4300343074024D0B40A00500BCE75F00AA42EFEA3E080EE8B
:20864000E0B46413E60886F030F708430720128803A6F018F68003B4750543070A8021B477
:2086600078054307108019B46F10430708801112874DF0A312874DA38095B4626243070299
:208680007A00C004C005C006C007AB0753031F7C00E60886F01287AFA6F018F6EDD007D0C3
:2086A00006D005D0042430B43A0040022407C0E00AE645F070CC12874DA902EF30E505744D
:2086C0002DF0A30A128756D0E0F0A3D9FA0808EF30E7A1EAC39E509C7420F0A30A80F4B484
:2086E000630DAA0112874D128756E6F0A380DEB47331C082C08386820886837A00E06004FF
:20870000A30A80F9868318868212874D12875612874DE0A312874D6004F0A380F2D005D0D8
:208720000480AAB4691B86017A00E76004090A80F912874D1287568601E76091F009A380AB
:20874000F8F97A0112874D128756E9809ECDC583CDCCC582CC22EE601A8FF020F715C00219
:20876000EAC39E500C742030F6027430F0A30A80EFD00222C82581C822C92581C97A0022C6
:20878000D083D082CF2581F581CFC082C08322CF2581F581CF2229F9E5F03AFA227C00CB63
:2087A00030E7011CCB2275F00030E70215F022C002C001AAF0F97E007D007F11C3E933F97A
:2087C000EA33FADF08F5F0E9D001D00222ED33FDEE33FEC3ED9BF5F0EE9C40E0ADF0FED384
:2087E00080DBBB000122C333C5F033C5F0DBF7221287F304700205F0221287FC14B4FF0242
:2088000015F0221287FCF4C5F0F4C5F0221288604029801E12886040227017801E128860AC
:2088200040107017800C128860501080051288746009E4F5F02212887460F7E4F5F0042240
:2088400012887440F680EB12887440EF70E480EB12887440DD70E480D912887450DD80D208
:20886000C39BC5F09C20E70720D207C345F02220D2F9D322C5F0C39C7003E5F09B2290F0AF
:2088800000E0A360F8E0FFA3E0A3CF2582F582EF3583F58380EBFBE0CB22FCE0FBA3E0CC93
:2088A00022FAE0F9A3E0CA22AE88D388D7880A0A4469676974616C20436C6F636B2075737E
:2088C000696E67204453313330372049324320525443000A3E3E000A0A48454C50204D457C
:2088E0004E55202020202020202020202020202020200A2F207072696E742074696D652060
:208900002020202020202020202020202020200A74207365742074696D65202020202020FE
:20892000202020202020202020200A3F2068656C70000A20253032782D253032782D25300E
:20894000327820253032783A253032783A25303278000A656E7465722063757272656E7491
:118960002074696D652048483A4D4D3A5353203E0075
:00000001FF
